:020000040000FA
:10000000962A292053202820FF00030E8301A000F8
:100010000A08A1000408A200492800087F392C3CE6
:1000200000087F39031C2A3082073034F634A834A4
:10003000A434663425342134B634203424342234B4
:1000400061343934E03429342B346234FB34F034F5
:100050006B3479343234E334E1342A34EB342734EA
:100060006934F13470346434E634FF34BF34EF342F
:10007000FD34ED34AD342E34E934B4347234FD340F
:10008000FD34FD3474080339820720344034803451
:1000900020340B117408753E840086122A308505C1
:1000A00018308605F20B6F281030F20007308316E7
:1000B00086048312060806080608060806080608CD
:1000C00006080739F1008316F83086058312FD080B
:1000D000031DFD038316A008031DA0038312F30B69
:1000E0007228B0150D20C6398604801F06140D2015
:1000F00019398400841904158411040885044220E8
:10010000203986044220C0398504F40A7408023C70
:10011000031CF4012208840021088A00200E8300B9
:10012000FF0E7F0E09001330AA005F30A228A53011
:10013000A0288A30A0281230A0280B30A028013037
:100140006400AA01A900A90BA3282A080319080022
:100150006400AA03A3280108C039031DAB280800C6
:100160000530A3003011AB2086118316861183124F
:1001700097208316861583129B20861930159920A7
:10018000301D0800A30BB32808000830AD00AB20D9
:10019000861183168611CC28CD280000861583127F
:1001A0009F20D228031086190314B10C9D20AD0B9B
:1001B000C92831080800B1010230C628B100083052
:1001C000AD00AB208611B10C831686118312031C7F
:1001D0009B20EA2883168615831203189B209F20F4
:1001E000AD0BE32808000130E0283108AC000830EE
:1001F000AD00AC0C03180329B21B05290310B20D86
:10020000AD0BF9280800B21BFE281830B206031403
:10021000B20D00292830A4000830A300DB202408F8
:10022000B100F320A40CA30B0E290800B301AC010C
:10023000B020F030DE200A212C080B21DB2003192E
:100240003829C03A031931293308353E84002C0877
:100250008000B30A3308803EF5000F3033020318E4
:100260000800AC0F1829B508031D0800F7013A294A
:100270000230F700F6018E30F5000800FD08031D7E
:100280000800861D0800340833020318B929B0207D
:100290003019C029F030DE200A213308353E8400B1
:1002A00000080B213030A300DB200319C029C03A1D
:1002B0000319C0290301311B0130B100F320A30B46
:1002C0005429BE30DE20B201C520A600F520C5208D
:1002D000A700F5200730A300C520F520A30B6C294B
:1002E000B208031DC0290222A3002708A40002228D
:1002F0000222A3070318A40A2708A407230EF03834
:10030000A300240E0F38A305240E0F39A41BF038C8
:10031000A400033A031DA4292308523A031DA4296B
:100320000310330D533E84000008A300840A000824
:10033000A4003E30A6000330A7005F23031CC029A1
:100340005230A3000330A4000310330D533E840049
:1003500023088000840A240880003308443E840077
:100360008001B30A34083302031C08002D30FD005D
:100370000800B020CC30DE204430DE20B30108007D
:100380003308443E8400001D800AB1292308AC00D4
:100390002408AD002508AE00A301A401A501183072
:1003A000AF000310E421031CDA29A5002A08A400E9
:1003B0002908A300AF0BD2292C0DA9002D0DAA00EE
:1003C0002E0DAB0003110800AC0DAD0DAE0DA30D4D
:1003D000A40DA50D26082302A9000301031C01306A
:1003E0002707AB0103182B142402AA002B08031CB7
:1003F00001302807AB0103182B1425022B1803101A
:10040000AB0008000310A60DA70D26080800A300E6
:10041000433E84000019532A230384000310040D73
:10042000533E84000008A300840A0008A400B0130F
:10043000A41F202AB017A409A309A30F202AA40AE5
:10044000A501E830A6000330A700A801C6212908AD
:10045000FB006430A600A701C6212908FA000A3073
:10046000A600A701C6212908F9002308F800B01B3F
:100470004E2AFB08031D462A7A0803192030F5008E
:100480007908803EF6007808F70008007B08F50040
:100490007A08F6007908803EF70008002230FA0852
:1004A000031D472A3F2A0E30F5009930F6004330ED
:1004B0000402803EF70008006400031783127E08E0
:1004C0008D0083168C18622A8C130C1483120C086E
:1004D000031308006400031783168C186D2A831217
:1004E0008C007E088D0083168C130C158B135530F1
:1004F0008D00AA308D008C148B170C1183120313FE
:10050000080064007108073A031D892A3012B015EB
:1005100008000315B01D08001830301EF430F30039
:10052000711DF301B0113016031108008316E83075
:100530008F0000309B00433081002A308500183046
:10054000860000308C00831220308B00FE01343096
:1005500084005C228000FE0A840A0408433C0318DD
:10056000A92A0730F100F201F401B921861DB62A4B
:10057000FD018B170130FC003408013C0319F12AFE
:1005800008308316A00083122030F500F6007C08A6
:10059000F7008122031D1C2B8316A0088312031D64
:1005A000C92A08308316A00083122030F7007C0887
:1005B000F6008122031D1C2B8316A0088312031D45
:1005C000D92A08308316A00083122030F6007C0858
:1005D000F5008122031D1C2B8316A0088312031D26
:1005E000E92A4B308316A00083123E217C080722A3
:1005F0008122031D1C2B8316A0088312031DF52ADC
:10060000FC0A7C0834020318BC2ABA2A3012812260
:100610000319142B71190F2B711C312B1C2B711CFE
:10062000242BF11C2C2B062B7108073A031D062BDB
:100630003E217C080722062B2630F5000C30F60000
:100640007C08803EF700062BFC0A7C083402031865
:100650001C2B0130FC00BA2AFC0B1C2B3408FC00BC
:10066000BA2A64008030F5000D30F6001A30F70029
:10067000B501B601B701B801B901BA01BB01BC01AE
:10068000BD01BE01BF01C001C101C201C3011621EC
:100690001E30A3009320A30B4A2B75088E3A031932
:1006A000312B3308B40034308400FE0100086A2284
:1006B000FE0A840A0408433C0318562BBA2A24086D
:1006C00027068039270D031D0800A501A801EA218E
:1006D000AB080319AA080319A90803190310080095
:02400E005C3F15
:02401000FC3F73
:104200000100FF00FF00FF00FF00FF00FF00FF00B4
:10421000FF00FF00FF00FF00FF00FF00FF00FF00A6
:10422000FF00FF00FF00FF00FF00FF00FF00FF0096
:10423000FF00FF00FF00FF00FF00FF00FF00FF0086
:10424000FF00FF00FF00FF00FF00FF00FF00FF0076
:10425000FF00FF00FF00FF00FF00FF00FF00FF0066
:10426000FF00FF00FF00FF00FF00FF00FF00FF0056
:10427000FF00FF00FF00FF00FF00FF00FF00FF0046
:10428000FF00FF00FF00FF00FF00FF00FF00FF0036
:10429000FF00FF00FF00FF00FF00FF00FF00FF0026
:1042A000FF00FF00FF00FF00FF00FF00FF00FF0016
:1042B000FF00FF00FF00FF00FF00FF00FF00FF0006
:1042C000FF00FF00FF00FF00FF00FF00FF00FF00F6
:1042D000FF00FF00FF00FF00FF00FF00FF00FF00E6
:1042E00029005300280032003000310031002E0038
:1042F00030003200FF00FF00FF00FF00FF00FF0062
:00000001FF
